:030000000209658D
:0C096500787FE4F6D8FD7581760209ACBD
:1009F10050000000000000000000000000000000A6
:030A0100000000F2
:060D6C008F907F017E0064
:030D7200020C462A
:0D0D4800C2A7120D6CD2A6120D6EC2A6221B
:0D0D5500D2A7120D6CD2A6120D6EC2A622FE
:080AEA008F398B3A8A3B893CED
:100AF200E4F53DAF05EF3395E04F7006E53924800C
:100B02008004E53924C0FF120D48AB3AAA3BA93C48
:100B12001208B5FFFD3395E04D6010120D557401BA
:0B0B2200253CF53CE4353BF53B80DF53
:010B2D0022A5
:0A0B70008F228D238B248A2589260D
:100B7A007536007537007538278B398A3A893B856F
:100B8A00363C85373D85383E7B017A007900120B69
:100B9A00EC7536007537007538007B017A007900EC
:070BAA00AD23AF22020AEAAD
:100C1A007F38120D48120D6E7F0C120D48120D6EA0
:100C2A007F06120D48120D6E7F01120D48120D6ECD
:0C0C3A007F80120D487F017E00020D72C9
:100CFC008F0853080F530501AF05EF7004E508800A
:0C0D0C0004E50824404480FF120D48223A
:0A0D62008B09120CFCAF09020D55BD
:100A470074656D703A2532640068756D693A2532B0
:100A57006400257300535700253264636D005825E1
:100A6700644825644425645A0D0A0053657420744C
:100A7700656D7000483A25326420204C3A2532646F
:100A8700005365742068756D69005365742053576A
:030A97002020001C
:100A04000258000001740001570A01551E01541ECA
:100A14000153500176020175060173000171000152
:100A24005A00017200015600016F00025B000011C0
:100A34005D00000000000000000000000000000055
:020A44000000B0
:100C4600D3EF9400EE64809480401D7D6EEDFB33FF
:100C560095E0FAD3EB9400EA6480948040031D800B
:080C6600ECEF1F70DB1E80D8CB
:010C6E002263
:1005BA0020B72D30B703020787AF73EF3395E04FAB
:1005CA0060030207877573010574D3E57494067492
:1005DA008094804003E4F57430B70302078780F8FB
:1005EA0030B6030206BD30B603020787AF73EF3396
:1005FA0095E04F6003020787757301E57424FE6076
:10060A003214604814605B14607114700302069E11
:10061A00240560030206B50555AF55EF3395E0FE94
:10062A00D3EF9432EE6480948050030206B5E4F569
:10063A005580780557AF57EF3395E0FED3EF9432E4
:10064A00EE648094804064E4F557805F0553AF53AD
:10065A00EF3395E0FED3EF945AEE64809480404BDA
:10066A0080140554AF54EF3395E0FED3EF945AEE5D
:10067A00648094804035E4F55380300575AF75EF9A
:10068A003395E0FED3EF9408EE64809480401CE436
:10069A00F57580170576AF76EF3395E0FED3EF94C4
:1006AA0008EE648094804003E4F57630B6030207CE
:1006BA008780F830B50302076930B503020787AFB0
:1006CA0073EF3395E04F6003020787757301E57492
:1006DA0024FE602414603514604614605714606860
:1006EA00240570761555AF55EF3395E0C3648094B1
:1006FA0080506775553280621557AF57EF3395E0D2
:10070A00C3648094805053755732804E1553AF534B
:10071A00EF3395E0C364809480503F75535A803A12
:10072A001554AF54EF3395E0C364809480502B7511
:10073A00545A80261575AF75EF3395E0C3648094DB
:10074A0080501775750880121576AF76EF3395E0ED
:10075A00C364809480500375760820B52080FB20FE
:10076A00B41420B418AF73EF3395E04F700F636F72
:0E077A000120B40980FBE4F573F55BF55C2209
:10000E005389F0438901E4F58A758CDCC28DD2A93F
:05001E00D28CD2AF22DC
:03000B00020B2EB7
:100B2E00C0E0C0D075D000C006C007758A00758CB5
:100B3E00DC1205BAE57164017018E56F7014055A80
:100B4E00D3E55A941E74809480400C755A00B2B34B
:100B5E008005D2B3755A000572D007D006D0D0D01A
:020B6E00E03273
:100D180053877F75985053890F438920758BFD75CC
:0B0D28008DFDC2ABD28ED2AFC2AC2258
:100BB1008B258A268927AE02AF01EF4E602CC2AC8D
:100BC100EDD39400748094804020AF051DEF601A2E
:100BD100AB250527E527AA267002052614F9120878
:0B0BE100B5F5993099FDC29980E02223
:100CDF008B228A238924AE02AF01EF4E600E120DD4
:0D0CEF0033AD07AB22AA23A924120BB122BA
:03002300020D7E4D
:050D7E00C298C2993289
:100C9600C2A000D2A000E4FFFEEEC39408748094C4
:100CA600805012EF25E0FFC2A100A2A2E433420762
:050CB600D2A10E80E454
:010CBB002216
:100CBC00E4FEFDEEFB3395E0FAC3EB9408EA6480A6
:100CCC009480500CEF20E0010DEFC313FF0E80E376
:020CDC00AF0562
:010CDE0022F3
:10038200120C1A120D1875250075260075276E7548
:1003920028027B007A007970120788D2B37FC87E68
:1003A20000120C4675250075260075276E75280209
:1003B2007B007A00797012078812000ED3E57294DE
:1003C200327480948040F5E4F572E57460030205AE
:1003D2000EE5566401700EF5567F01120D487F64DA
:1003E2007E00120D72120C96120CBCEF3395E0F5E2
:1003F200588F5975250075260075276E7528027B62
:10040200007A0079701207887BFF7A0A794775278C
:1004120000857028E4FDFF120B707BFF7A0A795089
:10042200752700856E287D01E4FF120B707527FF8A
:1004320075280A75295C7BFF7A0A7959E4FD7F0CDD
:10044200120B707BFF7A0A795F8558278559287DC0
:10045200017F0C120B70AF57EF3395E0FEAD707C4D
:1004620000C3ED9FEE6480F87480984067AF55EF4B
:100472003395E0FED3ED9FEE6480F874809850547B
:10048200AF54EF3395E0FEAD6EC3ED9FEE6480F89E
:10049200748098403FAF53EF3395E0FED3ED9FEE6B
:1004A2006480F8748098502CAF76EF3395E0FEC3E9
:1004B200E5599FEE6480F8E5586480984016AF7560
:1004C200EF3395E0FED3E5599FEE6480F8E558647A
:1004D200809840057571018003E4F5717542FF75DE
:1004E200430A754465754500857046754700856EFB
:1004F2004885584985594A7B007A00795D12008205
:100502007B007A00795D120CDF0203BEE556700FA4
:100512007556017F01120D487F647E00120D72E54F
:100522007424FE601314603014602D14605A146039
:1005320057240560030203BE7BFF7A0A7972E4FD49
:10054200FF120AEA7BFF7A0A797BAF55EF3395E017
:10055200F5278F28AF57801E7BFF7A0A7988E4FD42
:10056200FF120AEA7BFF7A0A797BAF53EF3395E0F9
:10057200F5278F28AF54EF3395E0F5298F2A7D01B7
:10058200E4FF120B700203BE7BFF7A0A7991E4FD4D
:10059200FF120AEA7BFF7A0A797BAF75EF3395E0A7
:1005A200F5278F28AF76EF3395E0F5298F2A7D0165
:0805B200E4FF120B700203BE0E
:040D83007F0CDFFE04
:010D87002249
:080D75007F247ED9DEFEDFFCC5
:010D7D002253
:05000300007F14DFFE88
:0100080022D5
:100A9A00E4FEFCECC39408748094805040E4FD208A
:100AAA00B20F000DEDD394FA7480948040F17F6404
:100ABA0022E4FD120D8330B209EE25E0FE43060161
:100ACA008006EE25E0FE801230B20F000DEDD394C1
:0F0ADA00FA7480948040F17F64220C80B6AF06DE
:010AE90022EA
:060788008B228A23892464
:10078E00E4FDF529F9F52AFBFC00C2B200120D7545
:10079E00D2B200120D830030B2030208AF20B20FA6
:1007AE00000DEDD394FA7480948040F17FFF22E423
:1007BE00FD12000320B2FD000DD3ED94FA74809467
:1007CE008040037FFF22C2AF120A9A8F29120A9A23
:1007DE00A907120A9A8F2A120A9AAB07120A9AAC22
:1007EE0007D2AFAF01E5292FFFE433FEE52A75836B
:1007FE00002FFFE5833EFEAD03ED7A002FFFEA3EAC
:10080E00FEEC6F7001EE6012E5296464700302085D
:10081E00ACE52A646470030208ACE52864017050EC
:10082E00E52A75F00A842430AB22AA23A9241208E3
:10083E00CEE52A75F00A84E5F02430AB22AA23A96E
:10084E00249000011208E0E52975F00A842430ABEB
:10085E0025AA26A9271208CEE52975F00A84E5F007
:10086E002430AB25AA26A9279000011208E0803477
:10087E00D3E52A9432748094805029C3E529945F7D
:10088E0074809480501EAB22AA23A924E52A120854
:10089E00CEAB25AA26A927E5291208CE80067FFF12
:0608AE00227FFF227F0003
:0108B4002221
:10097100020382E493A3F8E493A34003F68001F217
:1009810008DFF48029E493A3F85407240CC8C33387
:10099100C4540F4420C8834004F456800146F6DF56
:1009A100E4800B01020408102040809009F1E47EEC
:1009B100019360BCA3FF543F30E509541FFEE4934B
:1009C100A360010ECF54C025E060A840B8E493A312
:1009D100FAE493A3F8E493A3C8C582C8CAC583CA3D
:1009E100F0A3C8C582C8CAC583CADFE9DEE780BEF5
:010A460000AF
:1008B500BB010689828A83E0225002E722BBFE0241
:0908C500E32289828A83E4932274
:1008CE00BB010689828A83F0225002F722BBFE0109
:0208DE00F32203
:1008E000F8BB010DE58229F582E5833AF583E8F04E
:1008F000225006E92582C8F622BBFE05E92582C8FA
:02090000F222E1
:10002600E54E2442F8E6054E22783F300702784234
:10003600E475F00112092F0208B52000EB7F2ED2DD
:10004600008018EF540F2490D43440D4FF30040BB2
:10005600EF24BFB41A0050032461FFE54F60021578
:100066004F0552E5527002055130070D783FE47591
:10007600F00112092FEF0208CE020C6F7403D207AB
:100086008003E4C207F54E8B3F8A408941E4F54F71
:10009600F551F552E54F60077F2012006180F57536
:1000A60050FFC201C200C202C203C205C206C20894
:1000B60012002FFF700D3007057F00120072AF523D
:1000C600AE5122B4255FC2D5C20412002FFF24D040
:1000D600B40A00501A75F00A784F30D50508B6FFF5
:1000E6000106C6A426F620D5047002D20380D924C0
:1000F600CFB41A00EF5004C2E5D204020272D20154
:1001060080C6D20080C0D20280BCD2D580BAD205C9
:1001160080B47F201200612002077401B54F0040B1
:10012600F1120026FF12006102009AD208D2068060
:1001360095120026FB120026FA120026F94A4B7089
:100146000679437A037BFF20022EE54F602A7E0064
:100156008E8275830012090260060EEE655070F0FD
:10016600C2D5EBC0E0EAC0E0E9C0E0EE1202B9D0C9
:10017600E0F9D0E0FAD0E0FB1208B5FF60AAEBC0C8
:10018600E0EAC0E0E9C0E0120061D0E02401F9D065
:10019600E03400FAD0E0FBE5500460DCD550D980AD
:1001A600877BFF7A0279B5D202809C79108002792A
:1001B60008C206C2088008D2D5790A8004790AC224
:1001C600D5E550047002F550E4FAFDFEFF12002654
:1001D600FC7B08200113120026FD7B1030000A125A
:1001E6000026FE120026FF7B20EC3382D592D550E6
:1001F60013C3E43000069FFFE49EFEE42001039D46
:10020600FDE49CFCE4CBF8C201EC700CCFCECDCC67
:10021600E824F8F870F38017C3EF33FFEE33FEEDF2
:1002260033FDEC33FCEB33FB994002FB0FD8E9EBD3
:10023600300105F8D0E0C448B201C0E00AEC4D4EEA
:100246004F78207B0070C2EAB5500040BCC0E01277
:1002560002BBD0F0D0E0200104C4C0E0C4B201C0AB
:10026600F012004AD0F0D5F0EB02009A12093F01D5
:10027600375301B15801084C01044201B54F01BD85
:0F0286004401BD49011D4301C35501A74601A70E
:100295004501A747036350010C2D01102E01332B97
:1002A500011423013120034C2A00CC480000012B06
:1002B5003F3F3F00790AA2D5200314300509B91044
:1002C500020404B9080104A2D52006025001042045
:1002D50002689202B54F005034C0E07F2030031908
:1002E5007F30A20272067205500F120312C202C2BB
:1002F50006C205C2087F30800F300503E9C0E01251
:100305000061300503D0E0F9D0E0B54FCC300517DA
:100315007F30B9100C1200617F583004077F788058
:1003250003B908031200613002057F2D0200617FC9
:10033500202008F87F2B2006F322920280CF286E1A
:10034500756C6C2900D2011200263001F8C20178C3
:100355004F30D50108F60200CC2D50434958120004
:10036500262403B405004001E490035E9312005275
:0D037500743A120052D203754F040201B118
:100D3300E4FFFE1208B5600C0FEF70010E09E970B5
:050D4300F20A80EF221E
:100BEC00853942853A43853B44EBC53CFBEAC53D20
:100BFC00FAE9C53EF97F0978451208B5F60809E906
:0E0C0C0070010ADFF4AB3CAA3DA93E02008253
:10090200BB010CE58229F582E5833AF583E02250AA
:1009120006E92582F8E622BBFE06E92582F8E222F4
:0D092200E58229F582E5833AF583E493220E
:10092F00FAE6FB0808E6F925F0F618E6CA3AF622C9
:10093F00D083D082F8E4937012740193700DA3A347
:10094F0093F8740193F5828883E47374029368605B
:06095F00EFA3A3A380DF5B
:100C6F00EFB40A07740D120C7A740A309811A89910
:100C7F00B8130CC2983098FDA899C298B811F630E5
:070C8F0099FDC299F59922BD
:00000001FF
